:04000000DDEF13F02D
:1000080000C016F001C015F06F0084FF17F06F00F4
:1000180088FF18F0390193AF16D0A3AF14D03C0E67
:10002800B76EB00EB66E1C4A1D2A000E006E1D502B
:10003800005C02E11C50090805E2BA76010E1A6E4E
:10004800000E1B6EA39FA3A782D093A780D01AECA3
:100058000FF000C0C1F13D01F9AB10D0F99B010EC2
:1000680002019525006E000E9621016E00C095F2E2
:1000780001C096F21AEC0FF000C0C1F13D01F9A7DA
:100088000FD0010E02019525006E000E9621016E1B
:1000980000C095F201C096F21AEC0FF000C0C1F151
:1000A8000101C1510D0A0BE0C1510A0A08E0020121
:1000B800B051000802E1AF517F0801E328D00201E6
:1000C800010E976F000E986FB10EAB25E16E020E10
:1000D800AC21E26E6F0087FFE1FF6F008BFFE2FF4C
:1000E800E66A39019397ABC2AFF2ACC2B0F2020133
:1000F800AB6BAC6BB051000802E1AF517F0804E272
:10010800020E976F000E986F3901949520D0020166
:10011800976B986BB10EAB25E16E020EAC21E26EC7
:100128006F0087FFE1FF6F008BFFE2FF600007F7BA
:10013800E6FFABC2AFF2ACC2B0F2010EAB25006E67
:10014800000EAC21016E00C0ABF201C0ACF2390167
:1001580094A121D0A4A11FD0010E0201A55D006EBB
:10016800000EA659016E00C0A5F201C0A6F2000E4D
:10017800A65D02E1010EA55D08E239019491B290F5
:10018800010E01012D6F000E2E6F3C0EB16EB00EE8
:10019800B06E3901A49196AD26D0A6AD24D0010E3B
:1001A80002015325006E000E5421016E00C053F267
:1001B80001C054F25451FD0802E15351E8080DE220
:1001C800536B546B010E01012B25006E000E2C2180
:1001D800016E00C02BF101C02CF1FF0EA56EF00ED0
:1001E800A46E3901A69D91A109D0A1A107D0010E45
:1001F80002012A6F000E2B6F3901A19116C000F081
:1002080015C001F060005FF0E1FF600063F0E2FFFD
:020218001100D3
:0C021A00000E3D01F9BF010E006E120045
:0C022600000E3D01E1BF010E006E120051
:04023200F9DF1200DE
:04023600F1DF1200E2
:10023A00FBDF005202E10000FBD760007BFDD2FD2C
:02024A001200A0
:10024C00F4DF005202E10000FBD760007BFDEAFD09
:02025C0012008E
:08025E005DC35EF3EBDF12004B
:080266005DC35EF3F0DF12003E
:08026E005DC35EF3E3DF120043
:080276005DC35EF3E8DF120036
:0E027E00550E3A01BF6FAA0EBF6FBF9112005E
:10028C00D250026ED29E0500FF6A0150FE6E0050E5
:08029C00FD6E02BED28E1200BD
:0E02A400550E3A01BF6FAA0EBF6FBF81120048
:1002B20059C304F0BC92026A036A800E0318006EEE
:1002C200800E005C02E1080E025C1FE2800E041444
:1002D200016E0150800A02E1BC8201D0BC922A0E5A
:1002E2000D6E0D2EFED7000004360490BC842A0E3B
:1002F2000D6E0D2EFED70000BC942A0E0D6E0D2E33
:0C030200FED70000024A032AD8D71200E0
:10030E00086A096A100E0C6E01340836093604505C
:10031E00085E0550D8A0053C095ED8B007D0045041
:10032E0008260550D8B0053C0926D890003601366F
:06033E000C2EEAD71200AC
:1003440060008FFAE1FF600093FAE2FF600067FD4E
:0E035400E6FFA1C200F0A2C201F096DF120087
:1003620003015951170802E2006A0ED35A51000ADA
:10037200D8A4B1D05C5301E081DF60D060006FFD92
:1003820000FAA5D060006FFD01FAA1D060006FFDF8
:1003920002FA9DD060006FFD03FA99D060006FFDF4
:1003A20004FA95D060006FFD05FA91D060006FFDF0
:1003B20006FA8DD060006FFD07FA89D060006FFDEC
:1003C20008FA85D060006FFD09FA81D060006FFDE8
:1003D2000AFA7DD060006FFD0BFA79D060006FFDE4
:1003E2000CFA75D060006FFD0DFA71D060006FFDE0
:1003F2000EFA6DD060006FFD0FFA69D060006FFDDC
:1004020010FA65D060006FFD11FA61D060006FFDD7
:1004120012FA5DD060006FFD13FA59D060006FFDD3
:1004220014FA55D060006FFD15FA51D060006FFDCF
:1004320016FA4DD060006FFD17FA49D003015951E9
:10044200000A9CE05951010A9DE05951020A9EE0BE
:100452005951030A9FE05951040AA0E05951050A73
:10046200A1E05951060AA2E05951070AA3E05951E5
:10047200080AA4E05951090AA5E059510A0AA6E05E
:1004820059510B0AA7E059510C0AA8E059510D0A1B
:10049200A9E059510E0AAAE059510F0AABE059518D
:1004A200100AACE05951110AADE05951120AAEE0FE
:1004B2005951130AAFE05951140AB0E05951150AC3
:1004C200B1E05951160AB2E05951170AB3E00301DB
:1004D2005C5301E0E6DE03015A51010AD8A451D16E
:1004E2005C5301E0CBDEA4D0600067FDC0FA45D1C9
:1004F200600067FDC1FA41D1600067FDC2FA3DD1DB
:10050200600067FDC3FA39D1600067FDC4FA35D1D6
:10051200600067FDC5FA31D1600067FDC6FA2DD1D2
:10052200600067FDC7FA29D1600067FDC8FA25D1CE
:10053200600067FDC9FA21D1600067FDCAFA1DD1CA
:10054200600067FDCBFA19D1600067FDCCFA15D1C6
:10055200600067FDCDFA11D1600067FDCEFA0DD1C2
:10056200600067FDCFFA09D1600067FDD0FA05D1BE
:10057200600067FDD1FA01D1600067FDD2FAFDD0BB
:10058200600067FDD3FAF9D0600067FDD4FAF5D0B8
:10059200600067FDD5FAF1D0600067FDD6FAEDD0B4
:1005A200600067FDD7FAE9D0600067FDD8FAE5D0B0
:1005B200600067FDD9FAE1D0600067FDDAFADDD0AC
:1005C200600067FDDBFAD9D0600067FDDCFAD5D0A8
:1005D200600067FDDDFAD1D0600067FDDEFACDD0A4
:1005E200600067FDDFFAC9D0600067FDE0FAC5D0A0
:1005F200600067FDE1FAC1D0600067FDE2FABDD09C
:10060200600067FDE3FAB9D0600067FDE4FAB5D097
:10061200600067FDE5FAB1D0600067FDE6FAADD093
:10062200600067FDE8FAA9D0600067FDE9FAA5D08D
:1006320003015B51000AD8B457D75B51010AD8B401
:1006420057D75B51020AD8B457D75B51030AD8B4C3
:1006520057D75B51040AD8B457D75B51050AD8B4AF
:1006620057D75B51060AD8B457D75B51070AD8B49B
:1006720057D75B51080AD8B457D75B51090AD8B487
:1006820057D75B510A0AD8B457D75B510B0AD8B473
:1006920057D75B510C0AD8B457D75B510D0AD8B45F
:1006A20057D75B510E0AD8B457D75B510F0AD8B44B
:1006B20057D75B51100AD8B457D75B51110AD8B437
:1006C20057D75B51120AD8B457D75B51130AD8B423
:1006D20057D75B51140AD8B457D75B51150AD8B40F
:1006E20057D75B51160AD8B457D75B51170AD8B4FB
:1006F20057D75B51180AD8B457D75B51190AD8B4E7
:1007020057D75B511A0AD8B457D75B511B0AD8B4D2
:1007120057D75B511C0AD8B457D75B511D0AD8B4BE
:1007220057D75B511E0AD8B457D75B511F0AD8B4AA
:1007320057D75B51200AD8B457D75B51210AD8B496
:1007420057D75B51220AD8B457D75B51230AD8B482
:1007520057D75B51240AD8B457D75B51250AD8B46E
:1007620057D75B51260AD8B457D75B51270AD8B45A
:1007720057D75B51280AD8B457D703015C5301E01D
:1007820090DDA8D003015AB102D0C29001D0C2803C
:10079200F9D003015AB102D0C29201D0C282F2D082
:1007A20003015AB102D0C29401D0C284EBD003013A
:1007B2005AB102D0C29601D0C286E4D003015AB126
:1007C20002D0C29801D0C288DDD003015AB102D052
:1007D200C29A01D0C28AD6D003015AB102D0C29CB9
:1007E20001D0C28CCFD003015AB102D0C29E01D037
:1007F200C28EC8D003015AB102D0C39001D0C380C7
:10080200C1D003015AB102D0C39201D0C382BAD07F
:1008120003015AB102D0C39401D0C384B3D00301FF
:100822005AB102D0C39601D0C386ACD003015AB1EB
:1008320002D0C39801D0C388A5D003015AB102D017
:10084200C39A01D0C38A9ED003015AB102D0C39C7D
:1008520001D0C38C97D003015AB102D0C39E01D0FC
:10086200C38E90D003015AB102D0C49001D0C4808B
:1008720089D003015AB102D0C49201D0C48282D07D
:1008820003015AB102D0C49401D0C4847BD00301C5
:100892005AB102D0C49601D0C48674D003015AB1B1
:1008A20002D0C49801D0C4886DD003015AB102D0DD
:1008B200C49A01D0C48A66D003015AB102D0C49C42
:1008C20001D0C48C5FD003015AB102D0C49E01D0C2
:1008D200C48E58D003015951000AD8B453D7595184
:1008E200010AD8B456D75951020AD8B459D7595126
:1008F200030AD8B45CD75951040AD8B45FD7595106
:10090200050AD8B462D75951060AD8B465D75951E5
:10091200070AD8B468D75951080AD8B46BD75951C5
:10092200090AD8B46ED759510A0AD8B471D75951A5
:100932000B0AD8B474D759510C0AD8B477D7595185
:100942000D0AD8B47AD759510E0AD8B47DD7595165
:100952000F0A81E05951100A85E05951110A89E0C4
:100962005951120A8DE05951130A91E05951140A52
:1009720095E05951150A99E05951160A9DE05951CD
:0A098200170AA1E0FF0E006E12003C
:0C098C00000E3D0177BF010E006E12004E
:100998004FC359F350C35AF351C35BF3010E03011C
:0609A8005C6FDBDC1200B5
:1009AE000301525303E1010E006E27D13D0173B7CF
:1009BE002FD023C154F324C155F325C156F326C1BC
:1009CE0057F3DDDF005224E10101235124112511DB
:1009DE0026111DE00301545155115611571110E106
:1009EE0060000FF8E1FF600013F8E2FF030EE66E01
:1009FE0001C200F002C201F042DC010E006EFDD019
:100A0E00010E0301545F000E555B565B575BD9D741
:100A1E0060004BFD6CFD4FC300F00036009000509F
:100A2E00010F3D016E6F738B23C154F324C155F337
:100A3E0025C156F326C157F33D01030E7915006EFD
:100A4E0024E1010123512411251126111DE003017A
:100A5E00545155115611571110E160000FF8E1FF76
:100A6E00600013F8E2FF030EE66E01C200F002C250
:100A7E0001F005DC010E006EC0D0010E0301545FC3
:100A8E00000E555B565B575BD7D7FC0E3D017917B1
:100A9E00030153B103D03D01739D02D03D01738D0F
:100AAE000301586B5251585D3EE223C154F324C1E9
:100ABE0055F325C156F326C157F33D0178B125D024
:100ACE00010123512411251126111EE00301545159
:100ADE0055115611571111E160000FF8E1FF60003A
:100AEE0013F8E2FF030EE66E01C200F002C201F03F
:100AFE0046EC01F0010E006E80D0010E0301545F32
:100B0E00000E555B565B575BD8D70301600043FD63
:100B1E00E1FF600047FDE2FF6F00ABF5E6FF504BD3
:100B2E00512B582BBFD7000E000A02E1000E5319AD
:100B3E0033E123C154F324C155F325C156F326C125
:100B4E0057F33D0179B525D001012351241125110B
:100B5E0026111EE00301545155115611571111E182
:100B6E0060000FF8E1FF600013F8E2FF030EE66E7F
:100B7E0001C200F002C201F046EC01F0010E006E5F
:100B8E003CD0010E0301545F000E555B565B575B64
:100B9E00D8D73D01799530D023C154F324C155F3F4
:100BAE0025C156F326C157F33D0173B725D0010178
:100BBE0023512411251126111EE003015451551104
:100BCE005611571111E160000FF8E1FF600013F8A4
:100BDE00E2FF030EE66E01C200F002C201F046EC27
:100BEE0001F0010E006E09D0010E0301545F000EDC
:0C0BFE00555B565B575BD8D7006A1200AD
:100C0A00086A080E0C6E003408360450085ED8B024
:0E0C1A0002D00826D89000360C2EF5D7120016
:100C28000B6A0A6A096A005004026F00D0FF09F0D3
:100C38006F00CCFF08F0015005026F00D0FF0BF0E9
:100C48006F00CCFF0AF000500502F3500926F4505B
:100C58000A22E86A0B2201500402F3500926F450D4
:100C68000A22E86A0B2208C000F009C001F00AC095
:080C780002F00BC003F01200B2
:100C800003014F51390806E3300E4F5D03E3010EB7
:080C9000006E01D0006A1200A1
:100C98000301526B60003FFDE9FF600043FDEAFF7E
:100CA8006F00B8FF51F35151000A10E051C359F3D6
:100CB800A2EC01F00301522B52514F25E96E000EB0
:0E0CC8005021EA6E6F00B8FF51F3EDD7120015
:100CD600BC904F0E0D6E0D2EFED7000000004FC3C8
:100CE60059F359EC01F050C359F359EC01F04FC3D5
:100CF60059F359EC01F051C359F359EC01F04FC3C4
:100D060059F359EC01F052C359F359EC01F04FC3B2
:100D160059F359EC01F053C359F359EC01F0350E70
:0A0D26000D6E0D2EFED7BC801200EA
:100D30000301525303E1010E006E29D13D0173B747
:100D400030D023C154F324C155F325C156F326C135
:100D500057F31CDE005225E1010123512411251116
:100D600026111EE00301545155115611571111E17E
:100D700060000FF8E1FF600013F8E2FF040EE66E7A
:100D800001C200F002C201F046EC01F0010E006E5B
:100D9000FED0010E0301545F000E555B565B575B9E
:100DA000D8D760004BFD6CFD4FC300F000360090BB
:100DB000600003F06EFD3D01738B23C154F324C129
:100DC00055F325C156F326C157F33D01030E79159E
:100DD000006E25E1010123512411251126111EE089
:100DE0000301545155115611571111E160000FF8CC
:100DF000E1FF600013F8E2FF040EE66E01C200F0AE
:100E000002C201F046EC01F0010E006EC0D0010EEE
:100E10000301545F000E555B565B575BD6D7FC0E43
:100E20003D017917030153B103D03D01739D02D0F9
:100E30003D01738D0301586B5251585D3EE26000D5
:100E400043FDE9FF600047FDEAFF6F00BBFF6BFD5C
:100E500023C154F324C155F325C156F326C157F3DA
:100E60003D0178BB25D00101235124112511261104
:100E70001EE00301545155115611571111E1600044
:100E80000FF8E1FF600013F8E2FF040EE66E01C206
:100E900000F002C201F046EC01F0010E006E77D0C6
:100EA000010E0301545F000E555B565B575BD8D7AC
:100EB0000301504B512B582BBFD7000E000A02E103
:100EC000000E531933E123C154F324C155F325C156
:100ED00056F326C157F33D0179B525D001012351C1
:100EE0002411251126111EE00301545155115611EC
:100EF000571111E160000FF8E1FF600013F8E2FF05
:100F0000040EE66E01C200F002C201F046EC01F0F0
:100F1000010E006E3CD0010E0301545F000E555BC4
:100F2000565B575BD8D73D01799530D023C154F338
:100F300024C155F325C156F326C157F33D0173B7BC
:100F400025D0010123512411251126111EE0030192
:100F5000545155115611571111E160000FF8E1FF7E
:100F6000600013F8E2FF040EE66E01C200F002C258
:100F700001F046EC01F0010E006E09D0010E0301F4
:100F8000545F000E555B565B575BD8D7006A120062
:100F90000301536B050E535D0AE253515125E16E77
:100FA000000E5221E26E200EE66E532BF3D7535102
:100FB0005125E16E000E5221E26EE66A530753514D
:100FC0005125546F000E5221556F0A0E046E000E0B
:100FD000056E4FC300F050C301F087EC01F008C06C
:100FE00000F009C001F0300E0026600053FDE1FF63
:100FF000600057FDE2FF600003F0E6FF0A0E046E9A
:10100000000E056E4FC300F050C301F087EC01F0F5
:1010100000C04FF301C050F3000E011802E1000EB2
:0C102000001801E102D05307CAD71200EB
:10102C00310EB26E3C0EB16EB00EB06E3FC3A5F277
:10103C0040C3A6F201012D6B2E6BB2803901A49135
:04104C009481120079
:101050000201086B680E03014F6F080E506F020EFD
:10106000516F010E526F010E536F62DE680E030165
:101070004F6F080E506F020E516F120E526F536B6E
:1010800096DC08C228F209C229F20AC205F20BC294
:1010900006F202010B510608D8A0066B0CC207F23B
:0A10A0000DC230F20EC231F2120050
:1010AA000301456B466B3FC347F340C348F3800EC9
:1010BA004019006E800E005C02E1000E3F5D0BE2FB
:1010CA00010E456F000E466F3F510008476F40C33F
:1010DA0048F3000E485747C34FF348C350F341C380
:1010EA0051F342C352F34FDF060E436F000E446FB3
:1010FA00000E006E4451005C02E1435100081AE2FE
:10110A0043514125E16E44514221E26E010E435D95
:10111A00006E000E4459016E00504125E96E0150DF
:10112A004221EA6E6F00BBFFE6FF010E435F000E2D
:10113A00445BDED7600007FDE1FF60000BFDE2FFC4
:10114A00200EE66E455146111AE0436B446B43513B
:10115A004125E96E44514221EA6EEE50200A03E12C
:10116A00434B442BF4D7010E435F000E445B4351BB
:10117A004125E16E44514221E26E2D0EE66E1200C7
:10118A003FC300F00032009E0032009E0032009EF3
:10119A000032009E600003FDE1FF600007FDE2FFF0
:1011AA00300E0024E66E010E03014025E16E000EAA
:1011BA004121E26E0F0E3F15006E300E00266F00C1
:1011CA0087FFE1FF6F008BFFE2FF600003F0E6FF9D
:1011DA00020E4025E16E000E4121E26E6F0087FF8C
:0C11EA00E1FF6F008BFFE2FFE66A1200DD
:1011F6006000FFFCF6FF600003FDF7FF600007FDDF
:10120600F8FF09006F00D4FF00F0005216E06000FE
:10121600FFFCF6FF600003FDF7FF600007FDF8FF27
:1012260009006F00D4FF5DF33BEC01F0010E0301F2
:0C1236003F27000E40234123DBD71200AD
:0C1242003FC34FF340C350F326DD120001
:10124E003FC308F240C309F2680E03014F6F080E48
:10125E00506F020E516F020E526F536B62DD120011
:0C126E006F00A0F701F001C000F01200BA
:10127A006000FFFCE9FF600003FDEAFF6F00B8FFB2
:10128A0041F3000E0301426F000E426F000E421935
:10129A0002E1200E411907E0000E421902E1090E8F
:1012AA00411901E003D03F4B402BE2D7436B446B1B
:1012BA00456B466B000E421902E12D0E411905E1FC
:1012CA00454B462B3F4B402B08D0000E421902E1FA
:1012DA002B0E411902E13F4B402B6000FFFCE9FF56
:1012EA00600003FDEAFF6F00B8FF41F3000E426F92
:1012FA00000E426F41C34FF3BEDC005218E043C3F5
:10130A0000F044C301F00A0E046E000E056E87DC7D
:10131A00300E415D026E000E4259036E02500024E7
:10132A00436F03500120446F3F4B402BD6D74551A2
:10133A00461108E043510008006E44C301F0000E54
:0E134A00015604D043C300F044C301F012006A
:10135800020E0C6E9D0E0D6E0D2EFED70C2EFCD7B8
:061368000000000012006D
:10136E000301406B3F5109081BE20A0E046E3FC396
:10137E0000F044DC00C040F300C040F34037409121
:10138E004037409140374091403740910A0E046EED
:10139E003FC300F033DC08C000F00050401302D011
:0A13AE003FC340F340C300F01200FB
:1013B8000D0E03015D6F3BEC01F00A0E03015D6F3A
:0613C8003BEC01F01200F5
:1013CE000B0E0C6E570E0D6E0D2EFED70C2EFCD77F
:0613DE00000000001200F7
:0A13E400050E0D6E0D2EFED712004F
:1013EE00020E0C6E080E0D6E0D2EFED70C2EFCD7B7
:0413FE0000001200D9
:101402003FC39DF240C39EF241C39FF242C3A0F28A
:1014120043C3A1F244C3A2F245C3A3F246C3A4F25A
:1014220047C399F248C39AF249C39BF24AC39CF25A
:101432004BC3A7F24CC3A8F24DC3A9F24EC3AAF202
:02144200120096
:10144400160E03014F6F506B130E516FCCEC04F06A
:10145400170E03014F6F010E506F250E516FCCEC28
:0414640004F012007E
:1014680003013F6B406B800E4019006E800E005CDC
:1014780002E1080E3F5D11E23F51010F4F6F506BC3
:10148800516B526B536B23DC6A0E0D6E0D2EFED71B
:0C149800000003013F4B402BE6D7120080
:1014A40003013F510308D8A03F6B40510308D8A063
:1014B400406BF00E3D01F21703013F513D01F21361
:1014C400300EF21340C300F0003600900036009056
:1014D40000360090003600900050F413F38F120091
:1014E4003901DD8B23C13FF324C140F325C141F30E
:1014F40026C142F33901DCBB23D00101235124115D
:10150400251126111CE003013F51401141114211E4
:101514000FE160000FF8E1FF600013F8E2FF020E34
:10152400E66E01C200F002C201F046EC01F013D0F5
:10153400010E03013F5F000E405B415B425BDAD763
:10154400040E3D01736F800E746F756B030E7B6F19
:08155400070E7A6F738F12007D
:10155C00130E03014F6F010E506F210E516FCCEC27
:10156C0004F0140E03014F6F010E506F220E516FD9
:10157C00CCEC04F0130E03014F6F506B210E516F26
:10158C00CCEC04F0140E03014F6F506B220E516F14
:0C159C00CCEC04F03A0162876289120076
:1015A8000301416B426B3FC303F040C304F03FC3E8
:1015B80005F040C306F060000FF0E9FF600013F08B
:1015C800EAFFEE50200A04E14151421101E115D031
:1015D800010E416F000E426F60000FF0E9FF6000DE
:1015E80013F0EAFF600017F0E1FF60001BF0E2FF74
:1015F8006F00BBFFE6FF054A062A03C001F004C0DE
:1016080002F0034A042A600007F0E9FF60000BF0CB
:10161800EAFFEE50000ACFE13FC300F040C301F0FB
:021628001200AE
:10162A000201AB6BAC6B000EAC5D02E17F0EAB5DF1
:10163A0018E2B10EAB25E16E020EAC21E26E6F002C
:10164A0087FFE1FF6F008BFFE2FFE66A010EAB2521
:10165A00006E000EAC21016E00C0ABF201C0ACF20C
:10166A00E2D7AB6BAC6BAD6BAE6BAF6BB06B976B22
:10167A00986B0101C16B3D01F289F96BFA6B390173
:04168A009387120030
:10168E000F0E03014F6F506B516B526B536B6BEC24
:10169E0006F0090E03014F6F506B516B526B536B7B
:1016AE006BEC06F00A0E03014F6F010E506F010E28
:1016BE00516F010E526F010E536F6BEC06F00B0E55
:1016CE0003014F6F070E506F070E516F070E526FCB
:1016DE00070E536F6BEC06F00C0E03014F6F010EED
:1016EE00506F010E516F010E526F010E536F6BEC66
:1016FE0006F02A0E0C6E8D0E0D6E0D2EFED70C2ED4
:10170E00FCD7000000000301326B336B800E3319DF
:10171E00006E800E005C02E1080E325D0BE24F6B34
:10172E00506B516B526B536B6BEC06F00301324BEB
:10173E00332BECD792DED00E0C6EC90E0D6E0D2E25
:0C174E00FED70C2EFCD70000000012009B
:10175A00520E0B6E2B0E0C6E000E0D6E0D2EFED75A
:0C176A000C2EFCD70B2EFAD7000012004A
:1017760066DE340E03013F6F1E0E406F000E416F92
:10178600000E426F760E436F020E446F5D0E456F7C
:10179600030E466FFF0E476FFF0E486F000E496F30
:1017A600000E4A6F360E4B6F020E4C6F000E4D6FD9
:0E17B600000E4E6F23DE3F6B406B71DE1200A3
:1017C40032C300F00032009E0032009E0032009EC0
:1017D4000032009E0A0E00026F00CCFF01F00F0ED3
:0C17E40003013215006E015000261200B7
:1017F000BB8A090E0B6E1E0E0C6EE40E0D6E0D2EC6
:10180000FED70C2EFCD70B2EFAD70000BB9A020E87
:101810000C6E3D0E0D6E0D2EFED70C2EFCD700006B
:101820000000016A026A800E0218006E800E050A2E
:10183000005C02E1A00E015C16E2BB8A0000000021
:10184000000000000000BB9A000000000000000043
:101850000000000000000000000000000000000088
:10186000014A022AE0D7BB9A020E0C6E730E0D6E6F
:0A1870000D2EFED70C2EFCD712003F
:10187A0009006F00D7FFE6FF0006FAE10106F8E16A
:02188A0012004A
:10188C00090E0B6E1E0E0C6EE40E0D6E0D2EFED799
:0C189C000C2EFCD70B2EFAD70000120017
:1018A80003013A6B3B6B386B396B6000CBFCE9FF8B
:1018B8006000CFFCEAFFEE500008D8B075D2600097
:1018C800CBFCE9FF6000CFFCEAFF300EEE5C356F21
:1018D800366B376B800E3719006E800E005C02E1A4
:1018E800080E365DD8B057D2E4D16000CBFCE9FFD2
:1018F8006000CFFCEAFFEE502D0A25E13451010AC1
:1019080022E136513825006E37513921016EC20E59
:101918000024E16E010E0120E26E990E3625E96E73
:10192800000E3721EA6E6F00A7FFE9FF6F00ABFFDB
:10193800EAFF6F0087FFE1FF6F008BFFE2FF6F0098
:10194800BBFFE6FF32D036513825006E37513921BA
:10195800016EC20E0024E16E010E0120E26E030E3C
:10196800026E35C300F0000E016E025005E000362D
:1019780000900136FF0FFAD7410E0026000E012213
:1019880036510024E96E37510120EA6E6F00A7FF37
:10199800E9FF6F00ABFFEAFF6F0087FFE1FF6F0011
:1019A8008BFFE2FF6F00BBFFE6FF9ED13651382563
:1019B800006E37513921016EC20E0024E16E010E0E
:1019C8000120E26E030E026E35C300F0000E016EB8
:1019D800025005E0003600900136FF0FFAD7410E9D
:1019E8000026000E012236510024E96E37510120ED
:1019F800EA6E6F00A7FFE9FF6F00ABFFEAFF6F0019
:101A080087FFE1FF6F008BFFE2FF6F00BBFFE6FF80
:101A18003451000A32E1010E0101C015016E015076
:101A2800000A2BE1030136513825006E3751392160
:101A3800016EC20E0024026E010E0120036E910E8B
:101A48003625D96E000E3721DA6E60000BF0E9FFFB
:101A580060000FF0EAFF6F0067FFD9FF6F006BFFB0
:101A6800DAFFDE50EE10006E60000BF0E1FF600060
:101A78000FF0E2FF600003F0E6FF03013451010AB2
:101A88002AE136513825006E37513921016EC20ED0
:101A98000024026E010E0120036EB10E3625D96EA8
:101AA800000E3721DA6E60000BF0E9FF60000FF0DE
:101AB800EAFF6F0067FFD9FF6F006BFFDAFFDE50A8
:101AC800EE10006E60000BF0E1FF60000FF0E2FF27
:101AD800600003F0E6FF08D136513825006E375113
:101AE8003921016EC20E0024E16E010E0120E26E62
:101AF800030E026E35C300F0000E016E025005E0C1
:101B0800003600900136FF0FFAD7B90E0026000EF6
:101B1800012236510024E96E37510120EA6E6F0028
:101B2800A7FFE9FF6F00ABFFEAFF6F0087FFE1FF48
:101B38006F008BFFE2FF6F00BBFFE6FF3451000A26
:101B480032E1010E0101C015016E0150000A2BE1BE
:101B5800030136513825006E37513921016EC20E06
:101B68000024026E010E0120036E090E3625D96E7F
:101B7800010E3721DA6E60000BF0E9FF60000FF00C
:101B8800EAFF6F0067FFD9FF6F006BFFDAFFDE50D7
:101B9800EE10006E60000BF0E1FF60000FF0E2FF56
:101BA800600003F0E6FF03013451010A2AE13651CF
:101BB8003825006E37513921016EC20E0024026E9D
:101BC800010E0120036EA10E3625D96E000E3721B5
:101BD800DA6E60000BF0E9FF60000FF0EAFF6F00BB
:101BE80067FFD9FF6F006BFFDAFFDE50EE10006E63
:101BF80060000BF0E1FF60000FF0E2FF600003F00F
:101C0800E6FF72D036513825006E37513921016E02
:101C1800C20E0024E16E010E0120E26E030E026E78
:101C280035C300F0000E016E025005E0003600904A
:101C38000136FF0FFAD7B90E0026000E01223651E1
:101C48000024E96E37510120EA6E6F00A7FFE9FF13
:101C58006F00ABFFEAFF6F0087FFE1FF6F008BFFAC
:101C6800E2FF6F00BBFFE6FF3451010A21E1365164
:101C78003825006E37513921016EC20E0024E16EFD
:101C8800010E0120E26EA90E3625E96E000E3721FD
:101C9800EA6E6F00A7FFE9FF6F00ABFFEAFF6F0076
:101CA80087FFE1FF6F008BFFE2FF6F00BBFFE6FFDE
:101CB8001BD0000E3B1902E1000E3A19D8B415D614
:101CC800000E3B1902E1010E3A19D8B46FD6000E86
:101CD8003B1902E1020E3A19D8B4FED6000E3B19A0
:101CE80002E1030E3A198EE03651010F4F6F180EBC
:101CF8003625006E000E3721016EC20E0024E96EF3
:101D0800010E0120EA6E6F00A7FFE9FF6F00ABFF2D
:101D1800EAFF6F00B8FF50F3100E3625006E000E74
:101D28003721016EC20E0024E96E010E0120EA6E11
:101D38006F00A7FFE9FF6F00ABFFEAFF6F00B8FF76
:101D480051F3080E3625006E000E3721016EC20EC3
:101D58000024E96E010E0120EA6E6F00A7FFE9FF7B
:101D68006F00ABFFEAFF6F00B8FF52F3C20E3625D3
:101D7800E96E010E3721EA6E6F00A7FFE9FF6F00D9
:101D8800ABFFEAFF6F00B8FF53F36BEC06F00301FB
:101D9800364B372B9FD5080E3827000E3923324B88
:0A1DA800332B3A4B3B2B81D5120080
:101DB200CA6A020E3A01406F830EC26EC294C29684
:101DC200C298BA86BA88BA84506BCB6AFF0EC36EC9
:101DD200FF0E516FC384C382C398BB98C39ABB9A48
:101DE2003E01BC6BB86BFF0ECC6E3A01606B900E7D
:101DF200C46E130E166F150EE66F170EE56F618F28
:101E0200618D618B618161836185628F629D629B5D
:101E1200629562936291C490C494BC94C492BC8251
:101E2200618B618161836185629B6295629362913C
:021E320012009C
:061E340037EC09F012007A
:101E3A006000D3FCF6FF6000D7FCF7FF6000DBFC14
:101E4A00F8FF09006F00D4FF00F000521FE06000A5
:101E5A00D3FCF6FF6000D7FCF7FF6000DBFCF8FF5D
:101E6A0009006F00D4FF00F06000CBFCE1FF6000C6
:101E7A00CFFCE2FF600003F0E6FF0301324B332B95
:101E8A00010E3427000E35233623D2D76000CBFC4F
:0C1E9A00E1FF6000CFFCE2FFE66A1200EE
:101EA60032C302F033C303F002C000F003C001F0F6
:101EB600024A032A600003F0E9FF600007F0EAFF28
:101EC600EE5201E0F1D703013251025C006E33514C
:0E1ED6000358016E010E005E000E015A12004C
:101EE400020E0301326F000E336FDCEC09F00301C4
:101EF400366B376B39019397B10E0201AF25E16E52
:101F0400020EB021E26E6F0087FFE1FF6F008BFFCE
:101F1400E2FFE66A000EB05D02E1160EAF5DD8B0D6
:101F2400D2D0000E006EB051005C02E1AF51130834
:101F3400D8B0C9D0020E0301346F000E356F020110
:101F4400B0510301355D04E10201AF510301345D79
:101F54003EE2B10E3425E96E020E3521EA6E6F00C1
:101F6400A7FFE9FF6F00ABFFEAFFEE503B0A2CE14D
:101F7400B10E3425E16E020E3521E26E6F0087FF4B
:101F8400E1FF6F008BFFE2FFE66AF80E36253A6F39
:101F9400010E37213B6FB10E32253F6F020E332104
:101FA400406F3DEC09F06000EBFCE1FF6000EFFCEA
:101FB400E2FF600003F0E6FF364B372B010E3425B9
:101FC400326F000E3521336F344B352BB8D7FBC13C
:101FD40038F3000E396FFDC1FBF1FCC1FDF138C3CC
:101FE400FCF1F8C107F2F9C130F2FAC131F2FBC1D8
:101FF40006F20101FB5106080BE20201066B110E09
:1020040003013F6F470E406F000E416FFBEC08F079
:10201400FCC105F2FDC129F20201086B286B096BB2
:10202400FDC13FF3B7EC09F000C00AF205C23FF36B
:10203400B7EC09F000C00BF206C23FF3B7EC09F0AD
:1020440000C00CF207C23FF3B7EC09F000C00DF278
:1020540030C23FF3B7EC09F000C00EF231C23FF3D7
:10206400B7EC09F000C00FF2680E4F6F080E506F06
:10207400020E516F070E526F536B98EC06F0070E69
:102084000201086F100E096F680E03014F6F080EEE
:10209400506F020E516F010E526F536B98EC06F0A5
:1020A400070E03013F6F100E406F27EC09F06F0E0F
:1020B40003013F6F470E406F000E416FFBEC08F0C9
:1020C400DCEC09F012D0020E03013F6F450E406FA5
:1020D400000E416FFBEC08F0890E03013F6F440EC4
:0C20E400406F000E416FFBEC08F0120092
:1020F00028EC08F005C23FF31A0E0301406F010EF1
:10210000416FC5EC08F03A0E01011C6F29C23FF384
:102110001D0E0301406F010E416FC5EC08F03A0E31
:1021200001011F6F28C23FF3200E0301406F010E13
:10213000416FC5EC08F00101226B07C23FF3110E9D
:102140000301406F010E416FC5EC08F02D0E010137
:10215000136F30C23FF3140E0301406F010E416F45
:10216000C5EC08F02D0E0101166F31C23FF3170EBA
:102170000301406F010E416FC5EC08F00101196BBE
:1021800003013251010A1DE1110E3F6F010E406F34
:1021900021EC09F0520E3F6F490E406F000E416F67
:1021A000FBEC08F01A0E03013F6F010E406F21ECAB
:1021B00009F0520E3F6F490E406F000E416FFBEC6D
:0421C00008F0120011
:1021C4000301376B33AF0BD0010E376F2D0E0201B5
:1021D400556F0301321F331F324B332B04D0376B3F
:1021E400200E0201556F32C300F033C301F00132F7
:1021F4000032019E01320032019E01320032019E02
:1022040001320032019E00C034F30A0E046E05EC64
:1022140006F00A0E046E05EC06F008C000F0300E5D
:102224000024016E01C056F20150300A03E102019C
:10223400200E566F02010A0E046E34C300F005EC42
:1022440006F008C000F0300E0024576F32C335F397
:1022540033C336F30F0E03013215006E33C301F09E
:10226400000E011600C035F301C036F3710E046E82
:10227400020E056E14EC06F000C038F301C039F309
:1022840038C335F339C336F32E0E0201586FE80E06
:10229400046E030E056E38C300F039C301F087ECF9
:1022A40001F0300E0024596F640E046E000E056EAA
:1022B40038C300F039C301F087EC01F00A0E046E54
:1022C400000E056E87EC01F008C000F009C001F0B3
:1022D400300E00245A6F5B6B5C6B5D6B560E030112
:1022E4003F6F020E406FD4EC0AF03751010A17E138
:1022F40034C300F0000E016EE80E046E030E056E8A
:1023040014EC06F0355100240101276F0301365106
:1023140001200101286F000E296F2A6F1AD034C3DF
:1023240000F0000E016EE80E046E030E056E14EC50
:1023340006F00301355100263651012200500008F1
:102344000101276F01C028F1000E2857000E296FE4
:042354002A6F1200DA
:102358008C0E0101EC6F090EED6F000EEE6F000E92
:10236800EF6FAE0EF06F090EF16F4F0EF26F030EA6
:10237800F36F300EF46F0D0EF56F4F0EF66F030E00
:0C238800F76FAEEC0AF072EC0AF01200E5
:1023940015EC0BF032C33FF333C340F316EC08F0F3
:1023A400CE0E03013F6F460E406F000E416FFBECF3
:1023B40008F032C33FF333C340F3550E0301416FBA
:1023C400020E426F55EC08F0550E3F6F020E406F3F
:1023D400D4EC0AF0550E3F6F020E406F21EC09F069
:1023E400E70E3F6F480E406F000E416FFBEC08F0A4
:1023F400000E0201981902E1000E971908E1000E7F
:1024040001012E1902E1000E2D1901E1F1D701019C
:0E2414002D6B2E6B15EC0BF0DCEC09F01200BA
:10242200B28AB288B280B282320EB26EB36A010E42
:10243200B56E3C0EB16EB00EB06E3901A4918481BE
:102442000201A56BA66B01012D6B2E6BB2903901B7
:04245200949112004F
:10245600110E0301336F680E4F6F330E506F030E6C
:10246600516F010E526F536B98EC06F0680E030124
:102476004F6F330E506F030E516F020E526F536B38
:10248600D7EC04F033C33CF334C33DF3200E030111
:102496003E6F3CAF0AD02D0E3E6FFF0E3C1B3D53E8
:1024A60002E13C2B01D03D8107D03C51630804E298
:1024B600640E3C5F310E3E6F3EC333F3300E3E6F0B
:1024C6003C51090804E23E2B0A0E3C5FF9D73EC395
:1024D60034F3300E3C25356F2E0E366F300E3C6FC2
:1024E600300E3E6F3D5310E03DBD03D0350E3C6FC0
:1024F6000BD0320E3C6F350E3E6F3DA101D03D7FB5
:102506003DAF02D0370E3C6F3CC337F33EC338F3C2
:102516003251000A03E1B00E396F02D0DF0E396F77
:10252600430E3A6F3B6B330E006E030E016E1200C4
:1025360032C300F00032009E0032009E0032009E40
:102546000032009E900E0024F66E480EF76E000EC6
:10255600F722000EF86E000EF82209006F00D4FF75
:1025660000F06000CFFCE1FF6000D3FCE2FF6000FA
:1025760003F0E6FF010E03013325E16E000E342160
:10258600E26E0F0E3215006E900E0024F66E480EA7
:10259600F76E000EF722000EF86E000EF822090004
:1025A6006F00D4FF00F0600003F0E6FF020E332553
:0C25B600E16E000E3421E26EE66A1200B5
:1025C200BB8A00000000000000000000BB9A00006F
:1025D20000000000000000000000000000000000F9
:0825E2000000000000001200DF
:1025EA00BB8A00000000000000000000000000009C
:1025FA000000000000000000BB9A0000000000007C
:0E260A000000000000000000000000001200B0
:1026180034C301F0010E006E015004E00036009052
:10262800FF0FFBD700C036F3001E6000CBFCE9FFAC
:102638006000CFFCEAFF0050EF16F80EE9260050C4
:10264800EF16E7EC09F003013651EF12F80EE95ED8
:10265800ACEC09F03651EF14356F3551000A000E15
:10266800D8A4010E356FE7EC09F035C300F012006D
:10267800060E0C6E300E0D6E0D2EFED70C2EFCD7EE
:04268800000012003C
:10268C0034C301F0010E006E015004E000360090DE
:10269C00FF0FFBD700C038F3001C0301376F366BFC
:1026AC006000CBFCE9FF6000CFFCEAFF356B3551D5
:1026BC00070824E33751EF16F80EE9263751EF16C9
:1026CC00F2EC09F03851EF12F2EC09F0F80EE95E79
:1026DC003851EF14006E0CE035C301F0010E006EA2
:1026EC00015004E000360090FF0FFBD7005036136A
:1026FC00F7EC09F0F7EC09F0352BD9D736C300F01D
:02270C001200B9
:10270E00800E0301336F3351000814E2335132153A
:10271E00016E0150000805E22A0E5D6F3BEC01F0E0
:10272E0005D0200E03015D6F3BEC01F00301333346
:06273E00339FE9D71200F1
:1027440034C301F0010E006E015004E00036009025
:10275400FF0FFBD700C038F3001E00C037F3600042
:10276400CBFCE9FF6000CFFCEAFF0050EF16F80E47
:10277400E9260301366B3651070816E336C300F029
:1027840035C301F0005004E00132019EFF0FFBD776
:102794003751EF1601A002D03851EF12ACEC09F01A
:1027A4003851EF12362BE7D7F80EE95EF7EC09F053
:0627B400F7EC09F0120031
:1027BA00ACEC24F03901DE6BDD6BDA8DDA8BDA9959
:1027CA00DA97DA95DA93DA913C01E58FE589E597AC
:1027DA00E585E593E5913901DF87DF95DF93DF91A1
:1027EA00DD6BDD8D3C01E58FE589E597E585E593B0
:1027FA00E591E697E695E693E691010E0101E36F0E
:10280A00000EE46FBC806E0070F719F01A6A1B6A3A
:10281A001C6A1D6AD9EC0EF0290E0B6E960E0C6E10
:10282A007F0E0D6E0D2EFED70C2EFCD70B2EFAD76F
:10283A00BC80BB9A3F0E0C6E550E0D6E0D2EFED748
:10284A000C2EFCD701012F6B306B000E305D02E1BC
:10285A00400E2F5D10E2550E2F25E16E020E30213B
:10286A00E26E6F0087FFE1FF6F008BFFE2FFE66A0F
:10287A002F4B302BEAD72F6B306B000E305D02E105
:10288A00500E2F5D10E2310E2F25E16E010E302120
:10289A00E26E6F0087FFE1FF6F008BFFE2FFE66ADF
:1028AA002F4B302BEAD7F8EC0BF0090E0B6E1E0EED
:1028BA000C6EE40E0D6E0D2EFED70C2EFCD70B2ED1
:1028CA00FAD70000640E0101B16F000EB26FBA9818
:1028DA002F6B306B000E305D02E1800E2F5D10E22F
:1028EA00310E2F25E16E010E3021E26E6F0087FF57
:1028FA00E1FF6F008BFFE2FFE66A2F4B302BEAD72E
:10290A00310EBC6F010EBD6F400E3D01F56F030E17
:10291A00F66FF28FBBEC0BF0340E03013F6F1E0E05
:10292A00406F000E416F000E426F760E436F020E2B
:10293A00446F5D0E456F030E466FFF0E476FFF0E25
:10294A00486F000E496F000E4A6F360E4B6F020E2B
:10295A004C6F000E4D6F000E4E6F01EC0AF0520ED6
:10296A000B6E2B0E0C6E000E0D6E0D2EFED70C2E5E
:10297A00FCD70B2EFAD7000039015B91DCEC09F089
:10298A00310E0101BC6F010EBD6FBC8047EC0BF02C
:10299A00DCEC09F0310E0101BC6F010EBD6F440E73
:1029AA0003013F6F480E406F000E416FFBEC08F0C9
:1029BA0001012F6B306B000E305D02E10A0E2F5DB4
:1029CA0025E2030E006E000E016E2FC104F030C125
:1029DA0005F014EC06F0200E0024E96E000E01202A
:1029EA00EA6E6F00A7FFE9FF6F00ABFFEAFF6F0017
:1029FA00B8FF3FF36F00B8FF40F36F00B8FF41F331
:102A0A00FBEC08F001012F4B302BD5D7DCEC09F099
:102A1A00DE0E03013F6F470E406F000E416FFBEC65
:102A2A0008F046EC0CF00101BE6BBF6BCA0E030145
:102A3A00326F3F0E336F346BEADD19DECA0E326F26
:102A4A003F0E336F346B330E356F77DE10DECA0EEE
:102A5A00326F3F0E336F346B14DE00C0C1F107DEF4
:102A6A00A00E3F6F480E406F000E416FFBEC08F05E
:102A7A000201556BC1C132F3550E0301336F020EC9
:102A8A00346F54DD550E3F6F020E406F21EC09F092
:102A9A00230E3F6F490E406F000E416FFBEC08F0AA
:102AAA0001012F6B306B000E305D02E1060E2F5DC7
:102ABA002EE2CA0E0301326F3F0E336F346BE1DD33
:102ACA0000C0C1F1D4DDB30E01012F25E16E010E64
:102ADA003021E26E6F0087FFE1FF6F008BFFE2FF9C
:102AEA00600007F7E6FF0201556BC1C132F3550ECC
:102AFA000301336F020E346F19DD550E3F6F020E5C
:102B0A00406F21EC09F001012F4B302BCCD71B0E63
:102B1A0003013F6F490E406F000E416FFBEC08F056
:102B2A00CA0E0301326F3F0E336F346BAADD00C049
:102B3A00C1F10201556BC1C132F3550E0301336F66
:102B4A00020E346FF3DC550E3F6F020E406F21EC1C
:102B5A0009F0DCEC09F06D0E03013F6F480E406F7F
:102B6A00000E416FFBEC08F0CA0E0301326F3F0EF4
:102B7A00336F346B4CDDCA0E326F3F0E336F346BDA
:102B8A00CC0E356FDADDCA0E326F3F0E336F346BFF
:102B9A00440E356FD2DD6BDDCA0E326F3F0E336FD6
:102BAA00346B35DDCA0E326F3F0E336F346BCC0E89
:102BBA00356FC3DDCA0E326F3F0E336F346BBE0EF4
:102BCA00356FBBDDCA0E326F3F0E336F346B59DD82
:102BDA0000C01EF0000E1F6ECA0E326F3F0E336F1A
:102BEA00346B4FDD00C003F0026A1E500224006EEF
:102BFA001F500320016E00C0BAF101C0BBF100C032
:102C0A0032F301C033F3E2EC10F0550E03013F6FCB
:102C1A00020E406FD4EC0AF0550E326F020E336F7B
:102C2A0053EC0FF000C0E5F101C0E6F1550E0024A7
:102C3A00326F020E0120336F4D0E346F490E356F1D
:102C4A00000E366F1DEC0FF0550E03013F6F020E9A
:102C5A00406F21EC09F0DCEC09F0DCEC09F0DCEC6B
:102C6A0009F0F00E03013F6F460E406F000E416FF0
:102C7A00FBEC08F0ACEC11F0090E0B6E1E0E0C6E9C
:102C8A00E40E0D6E0D2EFED70C2EFCD70B2EFAD7A6
:102C9A000000590E03013F6F480E406F000E416F4E
:102CAA00FBEC08F0A80E03013F6F470E406F000EC1
:102CBA00416FFBEC08F00E0E0201086F400E096F1F
:102CCA00680E03014F6F080E506F020E516F020E0D
:102CDA00526F536B98EC06F0010E01012F6F000E34
:102CEA00306F000E305D02E1200E2F5D10E2080EFB
:102CFA002F25E16E020E3021E26E6F0087FFE1FFA1
:102D0A006F008BFFE2FFE66A2F4B302BEAD7CD0E1E
:102D1A0003013F6F480E406F000E416FFBEC08F055
:102D2A00000ECCB0010E03015D6F300E5D273BEC47
:102D3A0001F0DCEC09F0CBB226D02E0E03013F6F76
:102D4A00460E406F000E416FFBEC08F00201086B63
:102D5A00500E096F590E0A6F140E0B6F020E0C6F8C
:102D6A00200E0D6F020E0E6F190E0F6F680E030103
:102D7A004F6F080E506F020E516F080E526F536B51
:102D8A0098EC06F009D07F0E03013F6F480E406FA2
:102D9A00000E416FFBEC08F0DCEC09F00101BE6BA0
:102DAA00BF6B000EBF5D02E1040EBE5DD8B083D0DA
:102DBA000201086B680E03014F6F080E506F020E76
:102DCA00516F010E526F010E536F98EC06F0680EA8
:102DDA0003014F6F080E506F020E516F070E526FAC
:102DEA00536BD7EC04F008C228F209C229F20AC2CE
:102DFA0005F20BC206F202010B510608D8A0066BB7
:102E0A000CC207F20DC230F20EC231F2060E0101F7
:102E1A002F6F000E306F000E006E3051005C02E121
:102E2A002F51000826E2080E2F25E96E020E3021E6
:102E3A00EA6E6F00A7FFE9FF6F00ABFFEAFF6F00C2
:102E4A00B8FF3FF3550E0301406F020E416FC5EC08
:102E5A0008F0550E3F6F020E406F21EC09F0090E83
:102E6A005D6F3BEC01F0010E01012F5F000E305B3C
:102E7A00D2D708C23FF3550E0301406F020E416FCD
:102E8A00C5EC08F0550E3F6F020E406F21EC09F0B9
:102E9A00DCEC09F0520E0B6E2B0E0C6E000E0D6E52
:102EAA000D2EFED70C2EFCD70B2EFAD700000101EF
:102EBA00BE4BBF2B76D7320E03013F6F470E406FD2
:102ECA00000E416FFBEC08F00301326B2BEC12F0A1
:102EDA0000C03FF301C040F321EC09F0DCEC09F03B
:102EEA00520E0B6E2B0E0C6E000E0D6E0D2EFED7B3
:102EFA000C2EFCD70B2EFAD70000D76AD66A080E1A
:102F0A00D56EC60E03013F6F440E406F000E416F2F
:102F1A00FBEC08F0370E03013F6F450E406F000EC1
:102F2A00416FFBEC08F011EC12F0FE0E03013F6F4B
:102F3A00450E406F000E416FFBEC08F0D28E230E57
:102F4A0003015D6F3BEC01F0DCEC09F0640E030158
:102F5A00326F000E336FCAEC11F03F0E03015D6F42
:102F6A003BEC01F0DCEC09F00101E56BE66BCBB45C
:102F7A0042D1DCEC09F001012F6B306B000E305DA1
:102F8A0002E10A0E2F5DD8B02DD16A0E03013F6F00
:102F9A00450E406F000E416FFBEC08F0300E010148
:102FAA002F2503015D6F3BEC01F0DCEC09F0010118
:102FBA00BE6BBF6B000EBF5D02E1080EBE5DD8B0EE
:102FCA0004D1C20EBE25E16E010EBF21E26E2FC1F1
:102FDA0000F030C101F00036009001360036009052
:102FEA000136003600900136410E0026000E0122FD
:102FFA00BE510024E96EBF510120EA6E910EBE2532
:10300A00D96E000EBF21DA6E6F00A7FFE9FF6F00CD
:10301A00ABFFEAFF6F0067FFD9FF6F006BFFDAFFB4
:10302A00DE50EE10006E6F0087FFE1FF6F008BFF2E
:10303A00E2FF600003F0E6FFC20EBE25E96E010E54
:10304A00BF21EA6E6F00A7FFE9FF6F00ABFFEAFF3F
:10305A006F00B8FF32F387EC13F0550E3F6F490E3D
:10306A00406F000E416FFBEC08F0320E0101BE25E5
:10307A00E16E020EBF21E26E2FC100F030C101F0F5
:10308A000036009001360036009001360036009076
:10309A000136B90E0026000E0122BE510024E96E47
:1030AA00BF510120EA6E090EBE25D96E010EBF215D
:1030BA00DA6E6F00A7FFE9FF6F00ABFFEAFF6F0050
:1030CA0067FFD9FF6F006BFFDAFFDE50EE10006E6C
:1030DA006F0087FFE1FF6F008BFFE2FF600003F0E4
:1030EA00E6FF320EBE25E96E020EBF21EA6E6F00C0
:1030FA00A7FFE9FF6F00ABFFEAFF6F00B8FF32F3EB
:10310A0087EC13F00101BE51010F03014F6F320E1C
:10311A000101BE25E96E020EBF21EA6E6F00A7FF0C
:10312A00E9FF6F00ABFFEAFF6F00B8FF00F000C0D5
:10313A0050F3910EBE25E96E000EBF21EA6E090E0C
:10314A00BE25D96E010EBF21DA6E6F00A7FFE9FF17
:10315A006F00ABFFEAFF6F0067FFD9FF6F006BFFDD
:10316A00DAFFDE50EE100301516F00C052F3C20EB7
:10317A000101BE25E96E010EBF21EA6E6F00A7FFAD
:10318A00E9FF6F00ABFFEAFF6F00B8FF53F36BEC88
:10319A0006F0D00E0C6EC90E0D6E0D2EFED70C2E3B
:1031AA00FCD700000000030E0B6E080E0C6E770EA3
:1031BA000D6E0D2EFED70C2EFCD70B2EFAD7DCEC9B
:1031CA0009F00101BE4BBF2BF5D6DCEC09F00A0E63
:1031DA000301326F000E336FCAEC11F001012F4B5D
:1031EA00302BCCD6DCEC09F0320E0301326F000E24
:1031FA00336FCAEC11F0DCEC09F05D0E03013F6F8E
:10320A00460E406F000E416FFBEC08F0D2800201BF
:10321A002A6B2B6B3901A1919181DCEC09F0CBB4BB
:10322A00F5D1AB0E03013F6F460E406F000E416FA2
:10323A00FBEC08F0070E0C6E3A0E0D6E0D2EFED743
:10324A000C2EFCD7000002012C6B2D6B800E2D1961
:10325A00006E800E005C02E1050E2C5DD8B0D4D160
:10326A00F8EC0BF00101BE6BBF6BE56BE66BBF516F
:10327A00E65D02E1BE51E55DD8B08DD157D1E1ECF2
:10328A0012F0E1EC12F0E1EC12F0E1EC12F0E1ECF8
:10329A0012F0E1EC12F0E1EC12F0F5EC12F0E1ECD4
:1032AA0012F0E1EC12F0E1EC12F0E1EC12F0E1ECD8
:1032BA0012F0E1EC12F0E1EC12F0E1EC12F0E1ECC8
:1032CA0012F0E1EC12F0E1EC12F0E1EC12F0E1ECB8
:1032DA0012F0E1EC12F0E1EC12F0E1EC12F052D152
:1032EA00E1EC12F0E1EC12F0E1EC12F0E1EC12F098
:1032FA00E1EC12F0E1EC12F0E1EC12F0F5EC12F074
:10330A00E1EC12F0E1EC12F0E1EC12F0E1EC12F077
:10331A00E1EC12F0E1EC12F0E1EC12F0F5EC12F053
:10332A00E1EC12F0E1EC12F0E1EC12F0E1EC12F057
:10333A00E1EC12F0E1EC12F0E1EC12F0E1EC12F047
:10334A0021D1E1EC12F0E1EC12F0E1EC12F0E1EC47
:10335A0012F0E1EC12F0E1EC12F0E1EC12F0E1EC27
:10336A0012F0E1EC12F0E1EC12F0E1EC12F0E1EC17
:10337A0012F0E1EC12F0E1EC12F0E1EC12F0E1EC07
:10338A0012F0E1EC12F0E1EC12F0E1EC12F0E1ECF7
:10339A0012F0E1EC12F0E1EC12F0E1EC12F0F5ECD3
:1033AA0012F0F0D0E1EC12F0E1EC12F0E1EC12F0E4
:1033BA00E1EC12F0E1EC12F0E1EC12F0E1EC12F0C7
:1033CA00E1EC12F0E1EC12F0E1EC12F0E1EC12F0B7
:1033DA00E1EC12F0E1EC12F0E1EC12F0E1EC12F0A7
:1033EA00F5EC12F0E1EC12F0E1EC12F0E1EC12F083
:1033FA00E1EC12F0E1EC12F0E1EC12F0E1EC12F087
:10340A00F5EC12F0BFD0E1EC12F0E1EC12F0E1ECD5
:10341A0012F0E1EC12F0E1EC12F0E1EC12F0E1EC66
:10342A0012F0F5EC12F0E1EC12F0E1EC12F0E1EC42
:10343A0012F0E1EC12F0E1EC12F0E1EC12F0E1EC46
:10344A0012F0E1EC12F0E1EC12F0E1EC12F0E1EC36
:10345A0012F0E1EC12F0E1EC12F0E1EC12F0E1EC26
:10346A0012F0F5EC12F08ED0E1EC12F0E1EC12F071
:10347A00E1EC12F0E1EC12F0E1EC12F0E1EC12F006
:10348A00E1EC12F0F5EC12F0E1EC12F0E1EC12F0E2
:10349A00E1EC12F0E1EC12F0E1EC12F0E1EC12F0E6
:1034AA00E1EC12F0F5EC12F0E1EC12F0E1EC12F0C2
:1034BA00E1EC12F0E1EC12F0E1EC12F0E1EC12F0C6
:1034CA00E1EC12F0E1EC12F05DD0E1EC12F0E1EC8B
:1034DA0012F0E1EC12F0E1EC12F0E1EC12F0E1ECA6
:1034EA0012F0E1EC12F0F5EC12F0E1EC12F0E1EC82
:1034FA0012F0E1EC12F0E1EC12F0E1EC12F0E1EC86
:10350A0012F0E1EC12F0F5EC12F0E1EC12F0E1EC61
:10351A0012F0E1EC12F0E1EC12F0E1EC12F0E1EC65
:10352A0012F0E1EC12F0F5EC12F02CD0000E0201D0
:10353A002D1902E1000E2C19D8B4A1D6000E2D19AE
:10354A0002E1010E2C19D8B4CBD6000E2D1902E1D6
:10355A00020E2C19D8B4F5D6000E2D1902E1030E6D
:10356A002C19D8B41FD7000E2D1902E1040E2C19FC
:10357A00D8B449D7000E2D1902E1050E2C19D8B47A
:10358A0073D7A3D76A0E0D6E0D2EFED70000010168
:10359A00E54BE62B6CD6090E0B6E1E0E0C6EE40E76
:1035AA000D6E0D2EFED70C2EFCD70B2EFAD700006F
:1035BA00480E03013F6F490E406F000E416FFBEC4E
:1035CA0008F0BEC14FF3BFC150F3550E0301516F4E
:1035DA00020E526FC8EC07F0550E3F6F020E406F95
:1035EA0021EC09F0DCEC09F00101BE4BBF2B000E07
:1035FA00BF5D02E13C0EBE5DD8A037D6ADEC0BF044
:10360A0002012C4B2D2B22D6DCEC09F0C30E030150
:10361A003F6F470E406F000E416FFBEC08F03D0113
:10362A00F86B800EF46F3901818BA18B3D01FA6B27
:10363A00390193878387D28EF8EC0BF015EC0BF0E7
:10364A00BB9A010E0301326F78EC10F028C232F3F4
:10365A00E2EC0BF000C0C0F1C0C12EF2000E020174
:10366A002F6F29C232F3E2EC0BF000C0EAF105C277
:10367A0032F3E2EC0BF000C0EBF1B00E3F6F480EF4
:10368A00406F000E416FFBEC08F00301326B2BEC2C
:10369A0012F000C03FF301C040F321EC09F0200E04
:1036AA005D6F3BEC01F03B0E03015D6F3BEC01F0FB
:1036BA00CA0E0301326F3F0E336F346B0CEC13F0FA
:1036CA00CA0E326F3F0E336F346BCC0E356FA2ECDD
:1036DA0013F0CA0E326F3F0E336F346B440E356FE0
:1036EA00A2EC13F03CEC13F0CA0E326F3F0E336FAC
:1036FA00346B0CEC13F0CA0E326F3F0E336F346B1F
:10370A00CC0E356FA2EC13F0CA0E326F3F0E336F38
:10371A00346BBE0E356FA2EC13F0CA0E326F3F0E39
:10372A00336F346B46EC13F000C01EF0000E1F6EB0
:10373A00CA0E326F3F0E336F346B46EC13F000C083
:10374A0003F0026A1E500224006E1F500320016E0D
:10375A0000C0BAF101C0BBF100C032F301C033F3BB
:10376A00E2EC10F0550E03013F6F020E406FD4ECED
:10377A000AF0550E326F020E336F53EC0FF000C091
:10378A00E5F101C0E6F1550E0024326F020E012068
:10379A00336F430E346F490E356F000E366F1DECD2
:1037AA000FF0550E03013F6F020E406F21EC09F036
:1037BA00DCEC09F00101C0A510D058C257F27F0E07
:1037CA000201586F596B550E0301326F020E336FA7
:1037DA00010E346F54EC0CF012D01AC155F21BC111
:1037EA0056F21DC157F21EC158F20201596B550E0D
:1037FA000301326F020E336F346B54EC0CF001018B
:10380A00C051000A18E1F80E03013F6F470E406FDE
:10381A00000E416FFBEC08F0F8EC0BF0BB9A050EBA
:10382A000B6E0F0E0C6EF10E0D6E0D2EFED70C2EBA
:10383A00FCD70B2EFAD7800E0101E419006E800E18
:10384A00005C02E1020EE35DD8B0ACD1E76BE86B35
:10385A0002012C6B2D6B57D1E1EC12F0E1EC12F066
:10386A00E1EC12F0E1EC12F0E1EC12F0E1EC12F012
:10387A00E1EC12F0E1EC12F0E1EC12F0E1EC12F002
:10388A00E1EC12F0E1EC12F0E1EC12F0E1EC12F0F2
:10389A00E1EC12F0F5EC12F0E1EC12F0E1EC12F0CE
:1038AA00E1EC12F0E1EC12F0E1EC12F0E1EC12F0D2
:1038BA00E1EC12F0E1EC12F052D1E1EC12F0E1ECA1
:1038CA0012F0E1EC12F0E1EC12F0E1EC12F0E1ECB2
:1038DA0012F0E1EC12F0F5EC12F0E1EC12F0E1EC8E
:1038EA0012F0E1EC12F0E1EC12F0E1EC12F0E1EC92
:1038FA0012F0E1EC12F0E1EC12F0E1EC12F0E1EC82
:10390A0012F0E1EC12F0E1EC12F0E1EC12F0E1EC71
:10391A0012F0E1EC12F0E1EC12F021D1E1EC12F03C
:10392A00E1EC12F0E1EC12F0E1EC12F0E1EC12F051
:10393A00E1EC12F0E1EC12F0E1EC12F0E1EC12F041
:10394A00E1EC12F0E1EC12F0E1EC12F0E1EC12F031
:10395A00E1EC12F0E1EC12F0E1EC12F0E1EC12F021
:10396A00E1EC12F0E1EC12F0E1EC12F0E1EC12F011
:10397A00E1EC12F0E1EC12F0F5EC12F0F0D0E1EC2F
:10398A0012F0E1EC12F0E1EC12F0E1EC12F0E1ECF1
:10399A0012F0E1EC12F0E1EC12F0F5EC12F0E1ECCD
:1039AA0012F0E1EC12F0E1EC12F0E1EC12F0E1ECD1
:1039BA0012F0E1EC12F0E1EC12F0F5EC12F0E1ECAD
:1039CA0012F0E1EC12F0E1EC12F0E1EC12F0E1ECB1
:1039DA0012F0E1EC12F0E1EC12F0F5EC12F0BFD0CB
:1039EA00E1EC12F0E1EC12F0E1EC12F0E1EC12F091
:1039FA00E1EC12F0E1EC12F0E1EC12F0E1EC12F081
:103A0A00E1EC12F0E1EC12F0E1EC12F0F5EC12F05C
:103A1A00E1EC12F0E1EC12F0E1EC12F0F5EC12F04C
:103A2A00E1EC12F0E1EC12F0E1EC12F0F5EC12F03C
:103A3A00E1EC12F0E1EC12F0E1EC12F0F5EC12F02C
:103A4A008ED0E1EC12F0E1EC12F0E1EC12F0E1ECD4
:103A5A0012F0E1EC12F0E1EC12F0E1EC12F0F5EC0C
:103A6A0012F0E1EC12F0E1EC12F0E1EC12F0E1EC10
:103A7A0012F0E1EC12F0E1EC12F0E1EC12F0F5ECEC
:103A8A0012F0E1EC12F0E1EC12F0E1EC12F0E1ECF0
:103A9A0012F0E1EC12F0E1EC12F0E1EC12F0E1ECE0
:103AAA0012F05DD0E1EC12F0E1EC12F0E1EC12F070
:103ABA00E1EC12F0E1EC12F0E1EC12F0E1EC12F0C0
:103ACA00F5EC12F0E1EC12F0E1EC12F0E1EC12F09C
:103ADA00E1EC12F0E1EC12F0E1EC12F0E1EC12F0A0
:103AEA00F5EC12F0E1EC12F0E1EC12F0E1EC12F07C
:103AFA00E1EC12F0E1EC12F0E1EC12F0E1EC12F080
:103B0A00F5EC12F02CD00201000E2D1902E1000E84
:103B1A002C19D8B4A1D6000E2D1902E1010E2C19C8
:103B2A00D8B4CBD6000E2D1902E1020E2C19D8B446
:103B3A00F5D6000E2D1902E1030E2C19D8B41FD7A1
:103B4A00000E2D1902E1040E2C19D8B449D7000E23
:103B5A002D1902E1050E2C19D8B473D7A3D7020187
:103B6A00800E006E800E2D19005C02E12C510408B3
:103B7A0002E22C6B2D6B2C4B2D2B0101E74BE82B12
:103B8A00C051010F016E026A000E0222800EE8196E
:103B9A00006E800E0218005C02E10150E75DD8A0B9
:103BAA005AD665D2E76BE86B0A0E046EEAC100F0DA
:103BBA0005EC06F008C000F000C031F31AD2E1ECBF
:103BCA0012F0E1EC12F0E1EC12F0E1EC12F0E1ECAF
:103BDA0012F0E1EC12F0E1EC12F0E1EC12F0E1EC9F
:103BEA0012F0E1EC12F0E1EC12F0E1EC12F0E1EC8F
:103BFA0012F0E1EC12F0E1EC12F0F5EC12F0E1EC6B
:103C0A0012F0E1EC12F0E1EC12F0E1EC12F0E1EC6E
:103C1A0012F0E1EC12F0E1EC12F0E1EC12F0E1EC5E
:103C2A0012F0E1EC12F0E1EC12F0E1EC12F0E1EC4E
:103C3A0012F0E1EC12F0E1EC12F0F5EC12F0E1EC2A
:103C4A0012F0E1EC12F0E1EC12F0E1EC12F0E1EC2E
:103C5A0012F0E1EC12F0E1EC12F0E1EC12F0E1EC1E
:103C6A0012F0E1EC12F0E1EC12F0E1EC12F0E1EC0E
:103C7A0012F0E1EC12F0E1EC12F0E1EC12F0E3D117
:103C8A00E1EC12F0E1EC12F0E1EC12F0E1EC12F0EE
:103C9A00E1EC12F0E1EC12F0E1EC12F0E1EC12F0DE
:103CAA00E1EC12F0E1EC12F0E1EC12F0E1EC12F0CE
:103CBA00E1EC12F0E1EC12F0E1EC12F0E1EC12F0BE
:103CCA00E1EC12F0E1EC12F0E1EC12F0E1EC12F0AE
:103CDA00E1EC12F0E1EC12F0E1EC12F0F5EC12F08A
:103CEA00B2D1E1EC12F0E1EC12F0E1EC12F0E1EC0D
:103CFA0012F0E1EC12F0E1EC12F0E1EC12F0F5EC6A
:103D0A0012F0E1EC12F0E1EC12F0E1EC12F0E1EC6D
:103D1A0012F0E1EC12F0E1EC12F0E1EC12F0F5EC49
:103D2A0012F0E1EC12F0E1EC12F0E1EC12F0E1EC4D
:103D3A0012F0E1EC12F0E1EC12F0E1EC12F0F5EC29
:103D4A0012F081D1E1EC12F0E1EC12F0E1EC12F0A8
:103D5A00E1EC12F0E1EC12F0E1EC12F0E1EC12F01D
:103D6A00E1EC12F0E1EC12F0E1EC12F0E1EC12F00D
:103D7A00F5EC12F0E1EC12F0E1EC12F0E1EC12F0E9
:103D8A00F5EC12F0E1EC12F0E1EC12F0E1EC12F0D9
:103D9A00F5EC12F0E1EC12F0E1EC12F0E1EC12F0C9
:103DAA00F5EC12F050D1E1EC12F0E1EC12F0E1EC9A
:103DBA0012F0E1EC12F0E1EC12F0E1EC12F0E1ECBD
:103DCA0012F0F5EC12F0E1EC12F0E1EC12F0E1EC99
:103DDA0012F0E1EC12F0E1EC12F0E1EC12F0E1EC9D
:103DEA0012F0F5EC12F0E1EC12F0E1EC12F0E1EC79
:103DFA0012F0E1EC12F0E1EC12F0E1EC12F0E1EC7D
:103E0A0012F0E1EC12F01FD1E1EC12F0E1EC12F049
:103E1A00E1EC12F0E1EC12F0E1EC12F0E1EC12F05C
:103E2A00E1EC12F0F5EC12F0E1EC12F0E1EC12F038
:103E3A00E1EC12F0E1EC12F0E1EC12F0F5EC12F028
:103E4A00F5EC12F0F5EC12F0E1EC12F0E1EC12F004
:103E5A00E1EC12F0E1EC12F0E1EC12F0E1EC12F01C
:103E6A00E1EC12F0E1EC12F0EED0E1EC12F0E1EC50
:103E7A0012F0E1EC12F0E1EC12F0E1EC12F0F5ECE8
:103E8A0012F0F5EC12F0F5EC12F0E1EC12F0E1ECC4
:103E9A0012F0E1EC12F0E1EC12F0E1EC12F0E1ECDC
:103EAA0012F0E1EC12F0E1EC12F0E1EC12F0E1ECCC
:103EBA0012F0E1EC12F0E1EC12F0E1EC12F0E1ECBC
:103ECA0012F0E1EC12F0F5EC12F0BDD0E1EC12F0D8
:103EDA00E1EC12F0E1EC12F0E1EC12F0E1EC12F09C
:103EEA00E1EC12F0E1EC12F0F5EC12F0E1EC12F078
:103EFA00E1EC12F0E1EC12F0E1EC12F0E1EC12F07C
:103F0A00E1EC12F0E1EC12F0E1EC12F0E1EC12F06B
:103F1A00E1EC12F0E1EC12F0E1EC12F0E1EC12F05B
:103F2A00F5EC12F0F5EC12F0F5EC12F08CD0E1ECB5
:103F3A0012F0E1EC12F0E1EC12F0E1EC12F0E1EC3B
:103F4A0012F0E1EC12F0F5EC12F0F5EC12F0E1EC03
:103F5A0012F0E1EC12F0E1EC12F0E1EC12F0E1EC1B
:103F6A0012F0F5EC12F0F5EC12F0F5EC12F0E1ECCF
:103F7A0012F0E1EC12F0E1EC12F0E1EC12F0E1ECFB
:103F8A0012F0E1EC12F0E1EC12F0F5EC12F05BD079
:103F9A00E1EC12F0E1EC12F0E1EC12F0E1EC12F0DB
:103FAA00E1EC12F0E1EC12F0E1EC12F0F5EC12F0B7
:103FBA00E1EC12F0E1EC12F0E1EC12F0E1EC12F0BB
:103FCA00E1EC12F0E1EC12F0E1EC12F0F5EC12F097
:103FDA00E1EC12F0E1EC12F0E1EC12F0E1EC12F09B
:103FEA00E1EC12F0E1EC12F0E1EC12F0F5EC12F077
:103FFA002AD003013151000AD8B4E1D53151010A5E
:10400A00D8B40DD63151020AD8B43AD63151030A7E
:10401A00D8B467D63151040AD8B494D63151050AB6
:10402A00D8B4C1D63151060AD8B4EED63151070AEE
:10403A00D8B41BD73151080AD8B448D73151090A24
:10404A00D8B475D7A5D70101E74BE82BC051010FAA
:10405A00016E026A000E0222800EE819006E800EBE
:10406A000218005C02E10150E75DD8A09DD5210E3F
:10407A000B6E780E0C6E980E0D6E0D2EFED70C2E52
:10408A00FCD70B2EFAD70000000E02012B1902E111
:10409A00000E2A1901E1F8D72A6B2B6B000E98192A
:1040AA0002E1010E9719D8A4BFD0BA98F30E030102
:1040BA003F6F480E406F000E416FFBEC08F0B10EE7
:1040CA0003013F6F020E406F21EC09F0DCEC09F0AE
:1040DA00B10E0201AD6F020EAE6F6000B7FAE9FFD2
:1040EA006000BBFAEAFFEE50550A3AE1140EAD251C
:1040FA00E96E000EAE21EA6E6F00A7FFE9FF6F00BE
:10410A00ABFFEAFFEE50230A2BE1BF0E03013F6F1C
:10411A00480E406F000E416FFBEC08F0B10E030130
:10412A003F6F020E406F21EC09F0DCEC09F072ECF3
:10413A000FF028EC08F028C232F3E2EC0BF000C0D2
:10414A00C0F129C232F3E2EC0BF000C0EAF105C279
:10415A0032F3E2EC0BF000C0EBF10201AD6BAE6B97
:10416A006000B7FAE9FF6000BBFAEAFFEE504D0AB9
:10417A0056E1010EAD25E96E000EAE21EA6E6F0022
:10418A00A7FFE9FF6F00ABFFEAFFEE503D0A47E1E8
:10419A00020EAD25E96E000EAE21EA6E6F00A7FF92
:1041AA00E9FF6F00ABFFEAFFEE50310A10E0020EA2
:1041BA00AD25E96E000EAE21EA6E6F00A7FFE9FF9A
:1041CA006F00ABFFEAFFEE50320A01E028D0020E80
:1041DA00AD25E96E000EAE21EA6E6F00A7FFE9FF7A
:1041EA006F00ABFFEAFF6F00B8FFE9F1300E010183
:1041FA00E95DE36FE46B000EE45BDB0E03013F6FE6
:10420A00480E406F000E416FFBEC08F0E9C15DF308
:10421A003BEC01F0DCEC09F00201AD6BAE6BF8ECA3
:10422A000BF00101E76BE86B800E006E800E020155
:10423A009819005C02E19751010802E215EC0BF0B3
:06424A0023EF1BF0FFD77B
:1049580010EE19F0160E006E020E016E500EF66E75
:0E496800420EF76E000EF86E3DEC0CF01200E1
:01425000006D
:0242510000006B
:02425300000069
:02425500000067
:104257006643002B4800B14300514700464400FC29
:1042670043001248008546009D4500CE45008C4717
:014277000046
:1042780070888898A8C888702060A020202020F81E
:104288007088083860C088F870880838080888700E
:1042980018284888F8080808F88080F80808C870BE
:1042A80078C080F088888870F8881830202020200E
:1042B800708888F888888870F88888F8080808F06E
:0842C8000001010000010100EA
:0842D0000000007C000000006A
:0842D8000000000000008080DE
:0842E000705077040404040788
:0842E8000000000000000101CC
:1042F0000E1111131519110E040C14040404041FDB
:104300000E1101070C18111F0E1101070101110EEA
:10431000030509111F0101011F10101F0101190ED2
:104320000F18101E1111110E1F110306080808089E
:104330000E11111F1111110E1F11111F0101011E6C
:08434000008080000080800075
:0943480030302F30302F303000EE
:0943510030303A30303A303000CF
:04435A00000000005F
:04435E00000000005B
:02436200000059
:02436400000057
:10436600204469726563746F7279203A433A5C5FE0
:104376004D696B726F435C5F4D657350726F6A6512
:1043860074735F4D696B726F435C486F726C6F67D5
:10439600655F416E6E6561755F36306C6564735F2F
:0B43A60031384632374B34320D0A002C
:1043B1002050726F6A6574203A486F726C6F67653E
:1043C1005F50494331384632374B34325F416E6E6C
:1043D1006561755F36306C6564735F345F4D617420
:1043E10072696365735F4D6178373231395F313995
:0B43F10030362E6D637070690D0A00FD
:1043FC0020536F75726365203A20486F726C6F673B
:10440C00655F50494331384632374B34325F416E29
:10441C006E6561755F36306C6564735F345F4D61DA
:10442C007472696365735F4D6178373231395F310E
:0A443C0039303631392E630D0A00C5
:1044460020436F6E66696720626974203A202050A7
:1044560031384632374B34325F466F73635F496E8D
:104466007465726E655F36344D687A2E636667735F
:10447600636820464F53433A36342E30204D487AEF
:034486000D0A001C
:1044890020553B32343B30383B31373B31383B33B5
:10449900363B3034232020706F757220323420412E
:1044A9006F75742032303137202031384833362047
:0D44B90030343D4A657564690D0A0D0A0036
:1044C600204269742042616E6720536F66742053E0
:1044D600504920205243323D436C6B202C524331CD
:1044E6003D446F757420205243303D4353202D3E8A
:0C44F600204D4178373231393A0D0A0070
:104502000D0A2052617070656C20666F726D617465
:1045120020646520636465203A2022553B4A4A3B69
:104522004D4D3B41413B48483B4D4D3B6A443B234B
:0545320022200D0A002B
:10453700205465737420696E746572727570742087
:1045470054696D6572312020323020782031303047
:10455700206D73656320736F697420327365632000
:034567000D0A003A
:10456A00204465636F6D70696C652063686966666F
:10457A007265204720262044206176656320736592
:10458A007061726174657572732044206574204786
:03459A00202000DE
:10459D00204D6F64652031203A206368616E676538
:1045AD006D656E7420646520636F756C6575722022
:1045BD00636861717565207365636F6E64650D0A5F
:0145CD0000ED
:1045CE00204D6F64652032203A206368616E676506
:1045DE006D656E7420646520636F756C65757220F1
:1045EE00636861717565204D696E7574650D0A009D
:1045FE00205465737420576169745F4B657962202E
:10460E002D3E202054696D656F7574206F72206386
:10461E00686172207265636569766564200D0A00B3
:10462E00496E697420646174612052544320706134
:10463E0072206465666175742C2061766563205204
:0F464E0054435F466F7263E9653D30200D0A00EB
:10465D0020496E697420496E74657272757074208C
:10466D005242302C2073796E6368726F2031487A14
:08467D0020525443200D0A00F5
:10468500205072655465737420416666696368617C
:104695006765203020E0203920736920205242329E
:0646A5003D30200D0A006B
:1046AB00205072655F5465737420506172636F752F
:1046BB00727320646573203630206C656473202020
:0346CB000D0A00D5
:1046CE00202E2E2E2057616974696E67204B6579F6
:1046DE00626F61726420546F75636820666F72201A
:0246EE003C008E
:1046F00020496E6974204932433120485720524383
:10470000333D53434C205243343D534441200D0A22
:0147100000A8
:104711000D0A45727265757220737572204A6F7544
:10472100722053656D61696E65206A532E200D0AF2
:014731000087
:104732002054656D706572617475726520696E745E
:0F47420065726E6520445333323331203D2000C1
:1047510020546573742050494331384632374B3405
:0E47610032202049324331204857200D0A00F3
:10476F0045637269747572652064616E732044537A
:0D477F00333233312E2E2E204F4B0D0A0009
:10478C00496E697420666F72636167652052544389
:0C479C00207369205242313D300D0A00AC
:1047A8002041637469766520736F7274696520535C
:0B47B80051573D31487A3A200D0A00AD
:1047C30020496E697420496E746572727570742025
:0B47D30055415254205258200D0A009E
:1047DE00205465737420536F6E6465204F575320B9
:0A47EE00445331384232300D0A0006
:1047F8000D0A2052415A20616E6E6561752036306F
:0A480800206C65647320200D0A0087
:104812002031384632374B34322055415254312000
:094822004453333233310D0A0016
:10482B00204D696B726F432070726F20372E3330BF
:09483B002042657461200A0D00A1
:104844000D0A2050726573656E746174696F6E2011
:054854003A200D0A00EE
:1048590020496E6974205254432044533332333112
:04486900200D0A0014
:10486D00204D657375726520445331384232303DA9
:02487D00200019
:10487F002052652D4C656374757265205254432028
:01488F000028
:104890003031323334353637383941424344454676
:1048A0002046616D696C7920436F6465203A200071
:0F48B0002054656D70204453333233313D200066
:0E48BF0052544320557064617465203A200005
:0E48CD00205254435F466F7263E9653D200040
:0C48DB004E6577204D6F6465203D200085
:0C48E70020782032356D53203E0D0A0071
:0C48F3000D0A205265E775203A0D0A00FE
:0A48FF004D657263726564692E0056
:0949090056656E64726564690074
:0949120044696D616E6368650083
:08491B0020204352433D20001F
:07492300204944313D200052
:07492A0053616D6564690033
:064931004D617264690093
:064937004C756E6469007E
:06493D004A657564690083
:05494300B0432020003C
:05494800206A3D200083
:05494D00B04320200032
:0349520020200022
:034955002020001F
:020000040030CA
:0A000000040825A70B3F9F0F010025
:0200000400F00A
:020000040121D8
:1000000033656D20486F726C6F676520416E6E6559
:100010006175203630206C65647320524742202B76
:10002000206574204D617472696365203478204DB9
:1000300061783732313920202020202020200A0DFD
:100040004A756C69656E20465245594552200A0D25
:100050003135206A75696E2032303139200A0D0041
:1000600076657273696F6E20312031384632364BB7
:1000700032320A0D00FFFFFFFFFFFFFFFFFFFFFF10
:1000800056657273696F6E20322050726F746F20E4
:1000900031384632374B3432200A0D00FFFFFFFF64
:1000A000FFFFFFFFFFFFFFFFFFFFFFFFFFFFFFFF60
:1000B000FFFFFFFFFFFFFFFFFFFFFFFFFFFFFFFF50
:1000C000FFFFFFFFFFFFFFFFFFFFFFFFFFFFFFFF40
:1000D000FFFFFFFFFFFFFFFFFFFFFFFFFFFFFFFF30
:00000001FF
